:02000000802A54
:080008008D00030883128E0035
:100010008F1A0C288B1834280B190F2843280B1122
:10002000C93081000F1827288F1C2B28061C3F2859
:100030008F194128100891008F150F110F128F1082
:100040000F108F1285118B128B100B164328061878
:100050003F280F103228031006180314900C920347
:1000600003198F148B104328E93081008B100B117A
:100070008B160B12083092000F148F1643280F15A1
:100080001F280F161F280E0883008D0E0D0E090065
:100090008207523465346134643479340D34003469
:1000A0004534723472346F3472340D340034523447
:1000B0006534613464347934203474346F342034DA
:1000C000703472346F346734723461346D340D348B
:1000D00000344534723472346F3472343A3420341C
:1000E00075346E346B346E346F3477346E34203440
:1000F00063346F346D346D3461346E3464340D3474
:1001000000345234653461346434793420347434C6
:100110006F342034733474346134723474340D3475
:100120003E3400345634643464343D34353456340B
:100130000D3400345634643464343D3456346C34F5
:100140000D3400345634643464343D3456346834E9
:100150000D3400344E346F347434203465346E34CE
:100160006F347534673468342034643461347434E3
:1001700061340D34003450344F34483450346934D1
:100180006334203430342E34393462340D34003446
:100190000F39820730343134323433343434353427
:1001A00036343734383439344134423443344434C7
:1001B000453446349C001C1BDF280F3908003730BB
:1001C0001C020F3908008F1DE32811088F118515B7
:1001D00008008F01232285018601061483018316FE
:1001E0008030810001308600043085008312103099
:1001F0008B002E222A228515080093004820FF3903
:10020000031908000621930A1308FE2894002322EC
:10021000030166000A3092000B1103140610C83067
:1002200081000B1D11290B11920303191E29940C37
:10023000031C1C2906140F2906100F290130660023
:100240002A220800E3200D3C031D222908008C000F
:100250000630960004308C08031D05303C2206153C
:1002600010309D00861503108611051D03149E0C89
:100270009F0C9D0B32299E0C9F0C3F308C08031D58
:1002800003019E0508008400000EC8200621000816
:10029000C8200621840A000EC82006210008C820B4
:1002A00006210800222120309700003098000630F7
:1002B000960000303C221A30722108000630960069
:1002C00006303C22980A0319970A0800413006219B
:1002D00017304321080043300621233043210D30DD
:1002E000062108008400840A0830960000083C2299
:1002F000840300083C22080003109B0D9A0D063071
:10030000960002303C221A307221063096000830E6
:100310003C220F220E303C2203109A0C9B0CA40AA4
:10032000080004309900E320A0000D3A0319A92920
:100330002008DA20A0000430A100A00EA00D9B0D23
:100340009A0DA10B9E29990B932922213F309A05E2
:1003500008009A1708001B081F06031D08001A084A
:100360001E0608000301A300A40091219A1BEB299B
:1003700023222608463A0319C8291708203A031DE4
:10038000C8291808073A031DC8296430A500E629C2
:1003900003012721AB21031DCE29E2292608463A75
:1003A0000319F0297C2119302406031DC829FF30C8
:1003B000A400E02903012721AB21031DCE295E21E2
:1003C0002A2208002408A500A507A5070319DA2991
:1003D0007C21A503E6290730FD206130FD200800BF
:1003E0000301F82103012721AB21031DD729DA29B5
:1003F0008C0003109B0D9A0D0630960002308C087D
:10040000031D03303C221A3072210630960008305A
:100410003C221D2203109A0C9B0CA40A08000B110D
:10042000C83081000B1D122A080095010F220F22EF
:100430000F220F22950B162A0800623095000F221A
:10044000950B1F2A08008F1A232A8B138B1B252A32
:10045000851108008B108B1785150800860106167C
:100460001522061286161522861206171522061365
:100470008617152286130800A20016089D00861113
:100480000611000000008615A20C031806150000D6
:10049000000086119D0B402A08008C007F309A00D6
:1004A000FE309B00063096000B308C080319093093
:1004B0003C221A307221063096003C22063096000B
:1004C00008303C221D220800443006211E30432102
:1004D0000D3006210800A301A40191219A1BEB29EC
:1004E0002322FF302721AB2103197D2AFF30F82179
:1004F000FF302721AB21031DD7295E212A220800C6
:10050000E9207230FD203830FD20E3208C000D3AC8
:100510000319832A22210C08733A0319962A0C081E
:10052000663A0319982A2030FD20832A4530992AFB
:100530004630A60006169801970105141D22851461
:100540000E30FD206621203006210030FD202608D7
:1005500006213E300621E3208C000D3A0319A22A21
:100560000C08723A031DB92A2221030127216422B3
:10057000A22A0C08703A031DC02AB2216B21A22ABC
:100580000C08633A031DC92A522166210D30062149
:10059000A22A0C08693A031DD02A22215E21A22A30
:1005A0000C08713A031DD72A22218510802A0C08D5
:1005B000353A031DE32A22210616861206138613F6
:1005C0004930FD20A22A0C086C3A031DEF2A222193
:1005D00086160612061386135130FD20A22A0C0837
:1005E000683A031DFB2A222106170612861286137B
:1005F0005930FD20A22A0C08653A031D032B222145
:1006000003014D22A22A0C08453A031D0B2B22217F
:10061000FF304D22A22A0C08523A031D152B22212D
:10062000FF3027219E016422A22A0C08503A031DA4
:100630001C2B6B226B21A22A22212030FD20A22A12
:02400E00F23F7F
:00000001FF
